:1000000000308A00342900000A108A100A11820781
:1000100028340C34013406343330840000080319CA
:1000200020280130A100A001A00B1428A10B132847
:100030004A30A000A00B1A2800000000800B1128F5
:10004000003407080F39BA00390EA000F030A005BF
:100050002008F0393A0487000614831606100000C1
:10006000831206108316061083120034B708031D8E
:100070003B2886103C288614831686108312B80EFF
:100080003808B9002120B80E3808B90021200D30F9
:10009000A000A00B492800341430B3000C200F300E
:1000A0008316870583128610831686108312061026
:1000B000831606108312AA012A08023C031C682832
:1000C0000230B3000C200330B9002120AA0A5C28BA
:1000D0000D30A000A00B6A280230B90021200D309D
:1000E000A000A00B7128AA012A08023C031C842846
:1000F0002A080420AB00B7012B08B80036200230D4
:10010000B3000C20AA0A74288A116D290130330229
:10011000B5003408023C031D8F284030B507350870
:100120008038B600B7013608B800362000343208EF
:100130000C3A0319A528063A0319AD28073A031902
:10014000B328053A0319B828BD28B7010130B80013
:1001500036200230B3000C20C9280130B300023031
:10016000B4008620C9280130B300B4008620C92815
:10017000B7011030B8003620C92832081F3C031CD4
:10018000C3280730B2050130B7003208B800362066
:10019000C92800340408B100AB1FD7282D30B200A5
:1001A00097208403AA09AB09AA0A0319AB0A2B0EEC
:1001B000F038AD00AD07E23EAE00323EB0002B0895
:1001C0000F39AE07AE07B007E93EAF00AF07AF0784
:1001D0002A0E0F39AF07B007AF0DB00DB009B00D43
:1001E0002A080F39B007AD0D0730AC000A30B00750
:1001F000AF03031CF728AF07AE03031CFB28AE07B1
:10020000AD03031CFF28AD07AC03031C03292C30EE
:1002100084000730310584073030040203192C298B
:100220000008A000031D1A29311A2A29B1191C2916
:1002300020301D290830B1003030A007AB01040880
:10024000AA002008AC002008B20097202A088400E9
:100250002C08A000840A0C290008A0003030A00758
:100260002008B2009720003484011F3083058316D4
:100270001F149F141F159F11FF308312A5008316B2
:100280001F109F101F119F1183121F139F1383169E
:100290009F1783121F149412A51225088316870036
:1002A000831225162508831687008312A5112508B9
:1002B000831687000030831294008316940001088F
:1002C000C73908388100831290010030A1009200E4
:1002D00000308316920083124C286430B3000C2047
:1002E0000830A1001F08C73921049F000230AA006E
:1002F000FA30B3000C20AA0B78291F151F197E298C
:1003000083161E088312A6001E08A7001F151F19BA
:10031000872983161E0883122602A8002708A90031
:100320001E08031C1E0FA9026430B3000C2001300C
:10033000B300B40086201030AA002030B20097200D
:10034000AA0B9D29A91FCA290530B3000230B400A9
:1003500086202030B20097200A3084002908AB00A4
:100360002808AA00CA202030B20097202030B2000E
:1003700097202808083CAA00AB012908031C290F74
:10038000AB022A08B3000130B40086202A30B20044
:100390009720EF290630B3000230B40086202030C9
:1003A000B20097200A3084002908AB002808AA0070
:1003B000CA202030B20097202030B20097202808B1
:1003C000083CAA00AB012908031C290FAB022A082C
:1003D000B3000130B40086202A30B200972086296D
:0203E0006300B8
:02400E00393F38
:00000001FF
